:020000020000FC
:10000000EFC98FC20000000025C000004DC10000F4
:10001000000050C1000000000000000002030406C0
:10002000080C101820304060800002030406080C01
:10003000101820304080FF000406080C10182030F3
:10004000406080A0C0000D0D0403060D050D0602E2
:10005000030202004FB662FD1EC070FF18C165FDAD
:10006000F8C00994C0919700C395C0939700C5E06C
:10007000C519B8F3D0919700CD1B98F3C8E7089441
:1000800083FDC795C4BDC52DCC2321F4C0E083FDFD
:10009000C0E8C4BD07C171FF03C09598AC98C09873
:1000A000C52D089483FDC795C4BDC09399006B7F8F
:1000B000C52DCF3F09F441C0C0919800C395C093AE
:1000C000980070FF35C09598AC98C0984FBE1895B1
:1000D0007860C091A000CC2391F0C0919800CA959F
:1000E000D091A000CD1B58F0777FC0919800D0919F
:1000F0009F00CD1B08F41CC02092980019C0959851
:10010000AC98C098C5E0CA95F1F7C0917500CA9542
:10011000C2FD09C0C1FD05C095FFAB9A95FD949A3B
:100120000EC0AD9A0CC095FF949A95FDAB9A07C08E
:100130009598AC98C0984FBE1895209299004FBEE4
:100140001895A5C0552021F095FF959A95FDC09A68
:10015000AC989DC0552009F0AC9A95FFC09895FDCC
:10016000959895C0552021F095FFC09A95FD959AD8
:1001700095FF959895FDC0988AC095FF949895FD38
:10018000AB9895FFAB9895FD9498C5E0CA95F1F7AB
:10019000552021F095FF959A95FDC09AAC9877C0AF
:1001A00095FF949895FDAB98AD98C5E0CA95F1F789
:1001B000552021F095FF959A95FDC09AAC9867C09F
:1001C000AD9895FF949895FDAB98C5E0CA95F1F769
:1001D000552009F0AC9A95FFC09895FD959857C0A9
:1001E000AD9895FFAB9895FD9498C5E0CA95F1F749
:1001F000552009F0AC9A95FFC09895FD959847C099
:1002000095FFAB9895FD9498AD98C5E0CA95F1F728
:10021000552021F095FFC09A95FD959A95FF9598E8
:1002200095FDC09834C095FFAB9895FD949895FFC7
:10023000949895FDAB98C5E0CA95F1F7552021F04B
:1002400095FFC09A95FD959A95FF959895FDC09854
:100250001EC082FF1CC0C0917500C2FD0BC0C1FD55
:1002600011C095FF949895FDAB9895FFAB9895FDBF
:1002700094980DC0C1FDF5CF95FF949895FDAB986E
:10028000AD9805C0AD9895FFAB9895FD9498C52D98
:10029000C095089483FDC795C4BDC0939900209272
:1002A000970064604FBE18954FB6C0E1C8BF6E7F1F
:1002B0004FBE18953FB68F7EABB7A074A211806178
:1002C000A0E0ABBFA9B7AE7FA9BF7894A0916600AC
:1002D000AA2349F0A92FAF7151F1A0916600AA9508
:1002E000A093660024C040E050E0A0B396FDA09526
:1002F000A2FD4FEF96FFA3E096FDA2E0A5BFAA27BF
:10030000A064AABF8D7FA0B396FDA095A2FD5FEF6C
:10031000451749F7A0E461FDA0936600A92FAF71CE
:1003200019F0A0E4A093660040938D008160A09135
:100330006700AA2331F0A0916700AA95A0936700F7
:1003400007C0A92FAF7121F08061AA27A064AABFBE
:1003500080FF30C0A0918D004A2F8E7FA92FAF71F2
:1003600009F000C04093610071FF08C0A0916100D6
:1003700050919200A51710F0509361004091AE008B
:100380004430C1F4A091610040916300A41B70F05F
:100390004091CF00A40B50F0A0916300A40FA09354
:1003A000630040F4AFEFA093630004C0A09161002C
:1003B000A0936300A52DA03408F06860A0916000B0
:1003C000A395A093600051F0F894A9B7A160A9BFCC
:1003D00084FF02C0A0E4ABBF3FBE189542E050913D
:1003E0006600552331F0A92FAF7119F45A95509337
:1003F0006600A0918D00A13018F0209290000DC0F1
:100400002092910020929A00A0919000AF5FA0935B
:10041000900018F0AFEFA0939000B0906100509161
:10042000AE00523049F466FF91F0A2E3BA1678F0BC
:10043000A0917F00A0936100533049F466FF39F02A
:10044000A2E3BA1620F0A091BA00A09361005091E7
:1004500062005B1521F010F05A9501C0539550933E
:1004600062004A95D1F650919A00539509F45A9535
:1004700050939A00A0919B00AA95A0939B0009F02D
:1004800046C0A1E0A0939B0045E0A0919C005A17B4
:10049000F0F1A0919D005A1728F441E0A3E0A09349
:1004A0009B0007C0A0919E005A1718F441E04093AA
:1004B0009B00D0909300C0906300DC14A8F0A09142
:1004C000AE00A430D9F066FD0FC0C09293005395E2
:1004D00019F0A0919C00A0939A00A1E0A0939B002A
:1004E000ACE3A093620013C0A0919300A40F20F48A
:1004F0005FEF5093930002C0A0939300A0919300EC
:10050000AF3F29F4AFEFA0939100A0939A00F89425
:10051000A9B7A160A9BF84FF02C0A0E4ABBF3FBEE2
:1005200018953FB64CB55DB58F7EABB7A074A211E0
:100530008061A0E0ABBFA9B7AE7FA9BF789481FD71
:1005400026C096FFA2E096FDA3E0A5BF8260A0B3FF
:1005500096FDA095A2FF05C04093640050936500EE
:10056000FDC096FFA3E096FDA2E0A5BFAA27A06468
:10057000AABF8D7FA92FAF7109F4E1C040E0A0B3FD
:1005800096FDA095A2FDDBC040938D00CEC096FFE6
:10059000A3E096FDA2E0A5BF8D7F61FF6BC096FF33
:1005A000A2E096FDA3E0A5BFAA27A064AABF82602F
:1005B0004093880050938900A09086004A19B0901B
:1005C00087005B09BB24A2E0EA2EA22C483CA0E0F5
:1005D0005A0730F4A0E1BA2EE22CAAE0AA2E27C0D6
:1005E0004836A1E05A0730F4A8E0BA2EE22CAFE07A
:1005F000AA2E1DC0403DA2E05A0730F4A4E0BA2E56
:10060000E22CAEE1AA2E13C0403AA5E05A0730F41E
:10061000A2E0BA2EE22CACE3AA2E09C04839A8E029
:100620005A0728F4A1E0BA2EE22CA8E7AA2EC42E7D
:10063000A0918A00CA1AD52EA0918B00DA0ADD207B
:100640002AF4AFEFC094D094CA1ADA0A20928C0030
:10065000CA14DE0418F4A1E0A0938C0040938A0031
:1006600050938B0040918800509189004093860000
:1006700050938700A09164004A1BA09165005A0B1B
:1006800094FD46C093FD44C092FD40C056954795E9
:1006900091FD3CC05695479590FD38C0D52EC42E8F
:1006A000D694C79461FD0CC0AC2DAC51AD2DA240C9
:1006B00008F045C0DD2021F4AC2DA85C08F43FC053
:1006C000A0E0EA2E97FD02C0E090C200AAEFEA0E79
:1006D000F22CF21CCE18DF084FB74170442319F0FA
:1006E00040E050E015C0AFEFCA16D20418F04FEF4B
:1006F00050E00EC0F090A700CF9C412D000C441F8D
:1007000050E008F012C04FEF50E00FC056954795EB
:1007100094FF07C0552309F04FEFA42FA6954A0F69
:10072000521D4F3F520508F04FEF40938D008160FE
:1007300061FF05C0AFE1A095A923AB299A2FA0E4E2
:10074000A0936600A92FAF7119F4AAE0A0936600E8
:1007500061FD04C0A92FAF7109F08F7EA0E2A093C4
:100760006700A92FAF7119F4AAE0A0936700F8946D
:10077000A9B7A160A9BF84FF02C0A0E4ABBF3FBE80
:10078000189511E00AC013E008C01AE006C01EE187
:1007900004C014E602C018EC00C005E1BB27BA95FE
:1007A000F1F70A95D9F71A95C1F708952AE338E7C2
:1007B00009C020E33CE806C02AE234EB03C025E28E
:1007C00038EC00C0652CB1E05B2E12E095FD9F7DFA
:1007D00095FF9062BB27AD98BA95F1F7552009F0C7
:1007E000AC9ABA95F1F7AC98BA95F1F7AD9ABA957B
:1007F000F1F7552021F095FF959A95FDC09AB0919B
:10080000A800BA95F1F795FF959895FDC098B7E8BF
:10081000BA95F1F71A95D1F6022FB22FBA95F1F7E2
:100820000A95D9F73A9571F6AD98562C0895221B82
:1008300039E0001F3A9509F40895221F211B18F48E
:10084000210F8894F6CF0894F4CF622C722CB0E07C
:100850008894B395221F331FE0F737952795889426
:10086000912E802E020B130B10F4192D082D10F46D
:10087000889401C00894661C771CBA9571F7172DEF
:10088000062D0895322D11232AF43A9500951095DE
:10089000031B130BF894029F712C002D129F912CB7
:1008A000802C7894780C172D921C292DB4E06B2E97
:1008B0002695179507956A94D9F7332321F000956B
:1008C0001095031B130B08950091AE00043009F43A
:1008D00074C0B0918D00B95198F0B72FB67081F403
:1008E00066FD2BC005E09090C000B92DBA9521F0AF
:1008F0000AE0BA9509F002E1B0917400B01BE0F093
:1009000066FF0AC0B0919500B0939300BFEFB0931B
:100910009A00B1E0B0939B00B0916100B093630086
:1009200020927700209278002092790020927A001D
:1009300020927B006F7B41C060649090C000B92D15
:10094000BA9579F4B0916200B095BB1FBB1F1B2F05
:10095000B7950B2FB12FB170B3951B2FB02FBE7F62
:1009600025C0B92DBA95BA9581F4B0916200B095C1
:10097000BB1FBB1FBB1F1B2FB7950B2FB12FB37016
:10098000B3951B2FB02FBC7F14C0B0916200B095FF
:10099000BB1FBB1FBB1FBB1F1B2FB7950B2FB12F3F
:1009A000B770B395B3951B2FB02FB87FB0540B2FF2
:1009B00012090093770010937800089566FF21C014
:1009C000109174001695009173000795B09177000F
:1009D000B01B0B2FB0917800B10B1B2F28F40038FF
:1009E000BFEF1B0740F009C00F37120508F405C020
:1009F0000FE710E002C000E81FEF00937C001093A7
:100A00007D00089566FF39C000917C00B0917900A7
:100A10000B0F10917D00B0917A001B1F20E03091E8
:100A20007D0033230AF42A95B0917B002B1F1AF422
:100A3000203F40F00AC02F3008F407C00FEF1FEF2F
:100A40002FE003C000E010E020EF30916300B09190
:100A500092003B1718F4332331F009C0B0917D00A8
:100A6000BB235AF004C0B0917D00BB2332F4009345
:100A7000790010937A0020937B00089566FF2FC0C1
:100A80002091CD0000917C00000F10917D00111F7E
:100A9000F9DE11232AF40038BFEF1B0740F009C02C
:100AA0000F37120508F405C00FE710E002C000E898
:100AB0001FEF002352F0B0916200B01B0B2F18F013
:100AC000013008F00AC001E008C000950F5FB09146
:100AD00062000B0F08F001C00FEF00937E00089535
:100AE00066FF2DC02091CE0000917A0010917B000E
:100AF000C9DE11232AF40130BFEF1B0740F009C003
:100B00000F3F120508F405C00FEF10E002C001E02E
:100B10001FEF112352F0B0917E00B01B0B2F18F085
:100B2000013008F00AC000E008C000950F5FB091E6
:100B30007E000B0F08F001C00FEF009363000895D3
:100B40000FEF677FB72FB670E9F46860B09174005B
:100B5000B83008F0677FB0917400A1F00FEF1091EA
:100B6000740065DEF894B09170000B9F112D002D7C
:100B70007894112309F00FEFB09195000B1710F442
:100B80000091950000939400089506D374FFB2E09D
:100B900074FDB1E0B7B9B6B1B068B064B6B9F1DD13
:100BA00074FFB2E074FDB1E0B7B9B6B1B068B0643B
:100BB000B6B9B6B1B6FDFDCF04B115B1B6B1BF77C8
:100BC000B6B923D324E72093A30030E03093A400E8
:100BD000732E7694622E6694620E731E262D372D28
:100BE0000217130778F08090A300B4E7B80DB09314
:100BF000A3008090A400B0E0B81DB093A400260D1F
:100C0000371DEECF8090A3009090A4001091A40017
:100C100016950091A300079516950795B091A3002E
:100C2000B00FB093A100B091A400B11FB093A20087
:100C300023E0169507952A95E1F72091AF002A95B4
:100C400029F42092A3002092A4000AC02A9521F042
:100C5000800E911E2A95E1F78092A3009092A40045
:100C600008952091AF00B6B1B6FDFBCF04B115B128
:100C7000B6B1BF77B6B9B091A500B395B093A50052
:100C8000B83060F12092A500B091CC00BB2321F1D7
:100C9000112329F0B091A600BF3F61F009C0B091C7
:100CA000A6000B1739F020F4BB2321F0BA9502C03F
:100CB000B395E1F300919200B093A600B83850F4D8
:100CC00000ECBD3738F400E8B23720F400E4B73662
:100CD00008F400E0009392007F7E0895213099F09F
:100CE0000F3FB3E01B0778F4B091A3000B17B0914E
:100CF000A4001B0740F4B0919200BB2359F0BA95B1
:100D0000B093920007C0B0919200BF3F19F0B39525
:100D1000B093920000919200B0916300B01B10F468
:100D200000916300B09193000B1750F00091930075
:100D3000B0919300BF3F21F0B0919300B093920027
:100D4000502EB091A500B73009F47061089502E308
:100D5000F894B091D0000B9F012D000C001F7894E7
:100D6000B09192000B1710F0009192000093610077
:100D700000936300502E0093950008952092730015
:100D8000B8E0B09374000895209180003091810004
:100D9000F8940CB51DB5200F311F3BBD2ABD616015
:100DA000B0E1B8BF78942091710030917200009347
:100DB000710010937200021B130B2091730030918D
:100DC0007400622E732EB4E08B2EB2E09B2EB09195
:100DD0007400B43010F08A949A94B83010F08A9469
:100DE0009A94769467948A94E1F7261937099920A2
:100DF00021F0169507959A94E1F7200F311F209363
:100E000073003093740008F00895BFEFB09373003F
:100E1000B093740008952091820030918300F8947B
:100E20000CB51DB5020F131F1BBD0ABD6160B0E1FB
:100E3000B8BF7894089560FDFECFEDDF0895B091BE
:100E4000BE0000916E00023808F0B395003A08F039
:100E5000B395B63008F0B5E09B2EBCE08B2EB09178
:100E60007400B33030F48394839482FF02C083947F
:100E70008394B23030F48394839482FF02C08394CD
:100E8000839471FF03C0B3E09B2E822C10917400F9
:100E90000091730024E0169507952A95E1F708194B
:100EA000120928F0B02FB250B12FB20910F402E0AD
:100EB00010E0312F202F712E602E76946794B92D7B
:100EC000B330E9F0B0FD05C0060D171D262D372DF6
:100ED00006C0000F111F0250120922E030E0B92DA8
:100EE000B33068F020938400309385000093800035
:100EF00010938100609282007092830008950093A5
:100F000084001093850020938000309381006092CC
:100F1000820070928300089560FDFECF20918200D0
:100F2000220F30918300331FB72FB67021F020912C
:100F3000730030917400F8940CB51DB5020F131FA7
:100F40001BBD0ABD6160B0E1B8BF789408956061CF
:100F50002092760020E004C060612092760020E2BA
:100F6000B72FB67009F06F7E789460FD05C0B09120
:100F70007600BB2309F0089501E063FF0AC0B09139
:100F80007400B33008F002E0B0917400B63008F09D
:100F900003E071FF01C006E060FD06C0B09176007D
:100FA000BB2311F0789408951AE083FF1AE0789437
:100FB00000000000F89462FD03C014E183FF14E117
:100FC00071FF01C018E7B4B530919900B31BB10BA4
:100FD00018F3B0917600B395B0937600B5E03B2F4F
:100FE0006B2E722CB8B1B072B21709F073943A95A7
:100FF000C9F77394761488F464FFB2CF6F7E3CB562
:101000006DB47090730080907400370D681C6BBCD9
:101010003ABD6160B0E1B8BFA3CF64FDA1CF0A952E
:1010200009F0BACF7894089571FF0AC0B0916D00AD
:10103000B395B0936D0060FD0CC020926D0009C0A7
:1010400060FD07C064FD05C067FD03C0BF91BF918F
:101050005DC408952091840030918500F8940CB50A
:101060001DB5020F131F1BBD0ABD6160B0E1B8BF03
:1010700078940895EFDF00E063FF03C064FF01C0D0
:1010800001E0F89410916E00B7E01B9F212D102D08
:101090007894200F269517952695179526951795E0
:1010A00010936E00183718F4B8E7B0936E000091F3
:1010B0006E00B0916F000B1720F060629598AC98AD
:1010C000C09860FDFECF0895F8949498AD98AB98C1
:1010D00082FF07C0E0E0F1E073FF03C0BEE1BA9514
:1010E000F1F795FF949A95FDAB9AB2E0B093750035
:1010F00089C0F89495FFC09895FD959882FF0DC022
:10110000E0EFF0E073FF0BC0AD9895FFAB9895FD55
:101110009498BEE1BA95F1F702C0EAEAF0E062FF06
:1011200003C0552009F0AC9AB3E0B09375006AC0D3
:10113000F8949498AD98AB9882FF07C0E0EEF0E089
:1011400073FF03C0BEE1BA95F1F795FFAB9A95FD29
:10115000949AB4E0B093750055C0F894AC9882FFAF
:101160000DC0E0EDF0E073FF0BC095FF949895FD86
:10117000AB98AD98BEE1BA95F1F702C0E2EAF0E0B3
:1011800062FF06C0552021F095FF959A95FDC09A03
:10119000B5E0B093750036C0F8949498AD98AB98CC
:1011A00082FF07C0EDEBF0E073FF03C0BEE1BA952C
:1011B000F1F7AD9AB6E0B093750024C0F89495FFAE
:1011C000959895FDC09882FF10C0E3E1F1E073FFB0
:1011D0000EC095FF949895FDAB9895FFAB9895FD43
:1011E0009498BEE1BA95F1F702C0E2EBF0E062FF3D
:1011F00006C0552021F095FFC09A95FD959AB1E063
:10120000B09375006F7D7894089521EA30E0F9017C
:101210009598AC98C0989498AD98AB986B7F0895CA
:10122000ACEAB0E007E00D9307E00D9301E00D9309
:1012300004E00D930FEF0D930D930BE00D9302E07F
:101240000D9301E00D9301E00D93A8EBB0E001E0F8
:101250000D9300E00D9304EB0D930FEF0D930D93A1
:101260000D9303E00D9301E00D9301E00D930FEF5B
:101270000D9305E20D9300ED0D9308E70D9308EC37
:101280000D9304E00D930DE00D9301E00D9300E04C
:101290000D930AE70D9307E00D9301E00D93089578
:1012A0002091BF0009E011E0223011F405E011E0C7
:1012B000233011F405E012E0243011F405E013E0CE
:1012C000253011F409E017E0263011F400E010E0B9
:1012D00000939F001093A0002091B3008B7F777F35
:1012E000B091B4009F7DB1FD90629F7BB091B5003D
:1012F000B1FD9064B22FB23011F0886001C0877FD9
:101300000895ECE1F0E00091AC000A95E00FF21DC9
:10131000B491B093CD000091AD000A95E00FF21D9D
:10132000B491B093CE0071DF0895EAE2F0E000914D
:10133000C7000A95E00FF21DB491B093CF0065DFAE
:101340000895E8E3F0E00091B2000A95E00FF21D85
:10135000B491B093D00059DF08950091CB000023E1
:1013600009F40395013108F001E1B02FB00FB00F7F
:10137000B0939C001B2FB10FB10FB00FB0939D0025
:10138000B10FB00FB00FB0939E000895B091C80098
:101390000FEF1CE0B23011F400EA1AE0B33011F4A0
:1013A00002E815E000936F0010937000089508950F
:1013B0002091C2003091C30097FF02C020E03FEFB0
:1013C000B32FB21B6B2EB25810F4B2E86B2E00E0B4
:1013D0000395609EB12DB058D8F30093A7000895EF
:1013E000F894E3E0F0E0B9E0B7BFB491B078C1F3AE
:1013F000F894A895B1B5B861B1BDB0E0B1BDB4E0A5
:10140000BEBFBFE5BDBF01DFB0E0B8BBB1E1B7BB58
:10141000B0E0B5BBB8E3B4BBB0E0B2BBB0E3B1BBC6
:101420002224A0E0B0E02D92AA31E9F7A0E6B0E0D6
:101430000FEF2D920A95E9F7F3DE8DD231DF61DFF0
:1014400074DF7FDF8ADFA2DFB2DFB2DF0091C4008A
:101450000093A800DADEB2E0B3BFB2E0BEBDB2E0F6
:10146000B5BDF89498D9A2D992D9A3D990D9A4D9C5
:101470008ED908D390D98FD98CD9B1E5B8BFB9BF6F
:10148000B0B7B860B0BFB6B1B460B6B97AD9789425
:101490007CDBB0E4BBBFBB27B064BABF8D7F7BD918
:1014A000B1E0B0936900626025E0B0918C00BB238D
:1014B00009F425E068D9B0918D00B230A8F3B92FB6
:1014C000BF7100918F0000938E00B0938F00B01712
:1014D00059F72A9551F76D7F96FFB3E096FDB2E07C
:1014E000B5BFBB27B064BABF8D7F53D94CD902E0DA
:1014F000B92FBF7109F400E0B0918D00B017B0F3BF
:10150000F89454D953D952D9789445D920927F0070
:101510003AD9B091B800B13008F46CC0B09169000C
:10152000B13008F467C0B92FBF71C1F0B0918D0020
:10153000BF3F08F45FC0F89442D978942AD9B0919B
:101540008D00B130C0F7F89431D91FD92FD97894D4
:1015500020D9B0918D00BF3FB0F3C6C2B8E09B2E3A
:101560009068F89425DF789414D9F8949F7720DF59
:1015700080908D00B0918D00BF37789408F442C000
:1015800000D9F8941CD978949A9451F7B82DB55095
:10159000B093C30000D9F8940BD279D27894BAE012
:1015A0009B2E9068F89404DF7894F3D8F8949F7792
:1015B000FFDE80908D00B0918D00BF37789478F772
:1015C000E0D8F894F3D8E1D8F1D878949A9449F710
:1015D000B82DBB5FB093C200DED8F894E9D166D2D3
:1015E0007894D7D8F894E4DE7894B0918D00BF3F1A
:1015F000C0F37AC200918D00B0917F000B1710F0FC
:1016000000937F00C6D801E0B091B400B35009F454
:1016100005E0B0918D00B01708F07ACFF894CFD8DC
:10162000CED8CDD87894B7D82092690020926A009D
:1016300020926B00B0916A00B395B0936A00BF3FEF
:1016400069F5B0916B00B395B0936B00B091C60093
:1016500009E1BA9559F002E3BA9541F00DE7BA9560
:1016600029F00AEFBA9511F020926B00B0916B004F
:10167000B017A0F0B0916B00BA95B0936B00B4EBCB
:10168000B0936A00B091C500B093A800F89497D8C1
:101690007894B091C400B093A8007BD876D8B0916C
:1016A0006600BB2321F4B92FBF7109F4FCCEB091C1
:1016B0008D00B63008F4BECF6CD8B0916600BB2365
:1016C00009F4F1CEF894A1DD20926100209262002D
:1016D00020926300522C7894B091B100B0939600A0
:1016E00020927700209278002092790020927A0050
:1016F00020927B002092A50060E070E020926E00B6
:101700003DDBB8E0B093A50070613BD874FFB2E058
:1017100074FDB1E0B7B9B6B1B068B064B6B9B6B1EE
:10172000B6FDFDCF04B115B1B6B1BF77B6B911237F
:1017300009F00FEF0093A60094DAB8E0B093A5008B
:1017400070618090B300B2E0B093B300A9DD8092E5
:10175000B300F894BFEFB0939200F9DAB091610052
:10176000B0939200B0939300B09394007894B1E05A
:10177000B0936100B09363005B2EB0939B00B09177
:101780009100B0939A007160726020926D0004DD48
:1017900015DDFADAF3DA53DB04C082DD2092A5000E
:1017A0007F7E95FFB6E095FDB0E0B7B9D5DB3CDCB8
:1017B00051DC8AD85FDC88DCE7DA3DDB40DBACDB80
:1017C000B7E0B7B9C4DB30DC45DCF8D8B9D952DCB6
:1017D00090DCDADA30DB33DB9FDB95FFB0E095FDA0
:1017E000B6E0B7B9B9DB20DC35DC0CD943DCA0DCD2
:1017F000CBDA21DB24DB90DB95FFB6E095FDB0E092
:10180000B7B9A5DB11DC26DC39D934DCA6DCBCDABF
:1018100012DB15DB81DBB7E0B7B99EDB05DC1ADC38
:101820005FD928DCB9DCB0DA06DB09DB75DB95FFB4
:10183000B0E095FDB6E0B7B98ADB74FFB2E074FDA5
:10184000B1E0B7B9B6B1B068B064B6B9EDDB02DCEF
:1018500011DCB4DC99DAEFDAF2DA03DA5DDB71FF7E
:1018600020C067FD1EC0B0919500B0939200B09368
:101870009300B0919100B0939A00B1E0B0939B00B7
:1018800014E624E1B0916D00B11728F07D7F7460FB
:1018900020936C0006C0B0918D00B13008F081CF6C
:1018A00035C072FF10C067FD0EC0B0916C00BA95D4
:1018B00011F47B7F72CFB0936C00B0918D00B1308A
:1018C00008F06FCF23C0B0919000B13058F0B091C4
:1018D0009500B0939300B0919100B0939A00B1E05D
:1018E000B0939B00B0919000BA3F80F4B92FBF71C4
:1018F00021F4B0916600BB2349F0B091740000EF71
:1019000067FF01C000E6B01708F44BCFF8947DDC08
:101910008090B300B2E0B093B300C2DC8092B30019
:10192000209261002092620020926300522C20924B
:1019300096007E7F789425D768DCB92FBF7129F493
:10194000B0916600BB2309F4AECDB091B900B130BF
:1019500008F0CCCD6BCEEDE0F0E023D0053A09F0F5
:101960001BC0EEE0F0E01DD00A3509F015C03AE0EA
:10197000ACEAB0E0E3E0F0E014D00D9331963A9594
:10198000D9F735E1A8EBB0E0EFE0F0E00AD00D9335
:1019900031963A95D9F702C043DC0AD0E4E2F0E090
:1019A0000895E199FECFEEBBFFBBE09A0DB3089519
:1019B0001ED03AE0ACEAB0E0E3E0F0E00D910FD0E9
:1019C00031963A95D9F735E1A8EBB0E0EFE0F0E0D9
:1019D0000D9105D031963A95D9F712D00895E19935
:1019E000FECF0DBBEEBBFFBBE29AE19A0895EDE09E
:1019F000F0E00FEFF4DFEEE0F0E00FEFF0DF08953E
:101A0000EDE0F0E005EAEBDFEEE0F0E00AE5E7DF2D
:101A100008953091A9000091AA00313011F400938B
:101A2000AC00323011F40093AD00333011F4009368
:101A3000AE00343011F40093C000353011F400933F
:101A4000AF00363011F40093B200373011F4009338
:101A5000BE00383011F40093C700393011F4009300
:101A6000BF003A3011F40093B3003B3011F40093FF
:101A7000C8003C3011F40093B4003D3011F40093E1
:101A8000B500089525E087D62A95E9F708958ED602
:101A900090D692D694D679D689D68BD68DD68FD637
:101AA00074D684D686D688D68AD6089588D684D623
:101AB00080D67CD66AD683D67FD67BD677D665D6B7
:101AC0007ED67AD676D672D608958090A900909068
:101AD000AA006CD66BD66AD658D68A94D1F76FD640
:101AE00054D69A94E1F70895F894D1DF7894CADF38
:101AF000C9DFB1E0B093A900B1E0B093AA00209291
:101B0000AB00F894E2DF7894B5E06B2E70908D0016
:101B100042D6B0918D007B16C9F7B13018F0BF3FA7
:101B200040F107C076DFF89443DFB1DFB8E0B1BD24
:101B3000A9DF6A9459F7B091AB00B395B093AB00AD
:101B4000B33008F4DECF9EDFB091AA00B395B09316
:101B5000AA00F894B091A900BA95E6E4F0E0EB0F82
:101B6000F21D049178940395B091AA00B01708F47F
:101B7000C6CF88DF87DFB091A900B395B093A900E5
:101B8000B091A900BE3008F4B7CF4ADBF89410DF5B
:061B9000B8E0B1BD77DFF3
:00000001FF
